******************************************************************************
                  TI ARM Linker PC v5.1.5                      
******************************************************************************
>> Linked Wed Jul 22 14:23:52 2015

OUTPUT FILE NAME:   <Flash.out>
ENTRY POINT SYMBOL: "_c_int00"  address: 000005c4


MEMORY CONFIGURATION

         name            origin    length      used     unused   attr    fill
----------------------  --------  ---------  --------  --------  ----  --------
  VECTORS               00000000   00000200  00000020  000001e0     X
  BOOT_LOAD             00000200   00001000  0000064c  000009b4  R  X
  FLASH_API             00001200   00001000  000009e4  0000061c  R  X
  FLASH0                00002200   00018000  000096c6  0000e93a  R  X
  FLASH1                00020000   00060000  00000000  00060000  R  X
  FLASH2                00080000   00080000  00000000  00080000  R  X
  FLASH3                00100000   00040000  00000000  00040000  R  X
  STACK                 08000000   00001ff0  00000000  00001ff0  RW  
  SRAM                  08002000   00020000  00000f24  0001f0dc  RW  


SEGMENT ALLOCATION MAP

run origin  load origin   length   init length attrs members
----------  ----------- ---------- ----------- ----- -------
00000000    00000000    00000020   00000020    r-x
  00000000    00000000    00000020   00000020    r-x .intvecs
00000200    00000200    0000064c   0000064c    r-x
  00000200    00000200    000003c4   000003c4    r-x boot_code
  000005c4    000005c4    00000288   00000288    r-x eabi_start
00002200    00002200    000096c8   000096c8    r-x
  00002200    00002200    00009318   00009318    r-x .text
  0000b518    0000b518    0000035e   0000035e    r-- .const
  0000b878    0000b878    00000050   00000050    r-- .cinit
08002000    00001200    000009e4   000009e4    r-x
  08002000    00001200    000009e4   000009e4    r-x flashAPI
080029e4    080029e4    00000540   00000000    rw-
  080029e4    080029e4    0000044c   00000000    rw- .data
  08002e30    08002e30    000000f4   00000000    rw- .bss


SECTION ALLOCATION MAP

 output                                  attributes/
section   page    origin      length       input sections
--------  ----  ----------  ----------   ----------------
.intvecs   0    00000000    00000020     
                  00000000    00000020     sys_intvecs.obj (.intvecs)

boot_code 
*          0    00000200    000003c4     
                  00000200    000003c4     sys_core.obj (.text)

eabi_start 
*          0    000005c4    00000288     
                  000005c4    00000288     sys_startup.obj (.text:retain)

flashAPI   0    00001200    000009e4     RUN ADDR = 08002000
                  00001200    00000008     Fapi_UserDefinedFunctions.obj (.text)
                  00001208    00000810     bl_flash.obj (.text)
                  00001a18    00000178     F021_API_CortexR4_BE.lib : Program.obj (.text:Fapi_issueProgrammingCommand)
                  00001b90    0000000a                              : Utilities.CalculateEcc.obj (.tramp.Fapi_calculateEcc.1)
                  00001b9a    00000002     --HOLE-- [fill = 0]
                  00001b9c    0000000a                              : FlashStateMachine.IssueFsmCommand.obj (.tramp._Fapi_issueFsmCommand.1)
                  00001ba6    00000002     --HOLE-- [fill = 0]
                  00001ba8    0000000c                              : Read.MarginByByte.obj (.tramp.Fapi_doMarginReadByByte.1)
                  00001bb4    0000000c                              : Async.WithAddress.obj (.tramp.Fapi_issueAsyncCommandWithAddress.1)
                  00001bc0    0000000c                              : FlashStateMachine.EnableMainSectors.obj (.tramp.Fapi_enableMainBankSectors.1)
                  00001bcc    0000000c                              : FlashStateMachine.SetActiveBank.obj (.tramp.Fapi_setActiveFlashBank.1)
                  00001bd8    0000000c                              : FlashStateMachine.InitializeFlashBanks.obj (.tramp.Fapi_initializeFlashBanks.1)

.text      0    00002200    00009318     
                  00002200    00002ccc     sys_selftest.obj (.text)
                  00004ecc    00000b2c     system.obj (.text)
                  000059f8    00000b04     bl_ymodem.obj (.text)
                  000064fc    00000a50     sys_vim.obj (.text)
                  00006f4c    00000930     pinmux.obj (.text)
                  0000787c    000007c4     spi.obj (.text:retain)
                  00008040    00000768     sci_common.obj (.text)
                  000087a8    0000074c     sci.obj (.text)
                  00008ef4    000006c8     bl_uart.obj (.text)
                  000095bc    00000634     esm.obj (.text)
                  00009bf0    00000300     sys_mpu.obj (.text)
                  00009ef0    000002dc     sys_vim.obj (.text:retain)
                  0000a1cc    00000260     F021_API_CortexR4_BE.lib : FlashStateMachine.InitializeFlashBanks.obj (.text:Fapi_initializeFlashBanks)
                  0000a42c    000001a4     notification.obj (.text)
                  0000a5d0    00000198     ecap.obj (.text:retain)
                  0000a768    0000017c     F021_API_CortexR4_BE.lib : FlashStateMachine.SetActiveBank.obj (.text:Fapi_setActiveFlashBank)
                  0000a8e4    00000158     esm.obj (.text:retain)
                  0000aa3c    00000150     sw_hw_ver.obj (.text)
                  0000ab8c    00000114     sys_pmu.obj (.text)
                  0000aca0    000000e8     dabort.obj (.text)
                  0000ad88    000000a4     adc.obj (.text:retain)
                  0000ae2c    0000009c     rtsv7R4_T_be_v3D16_eabi.lib : memcpy_t2.obj (.text)
                  0000aec8    00000098     gio.obj (.text:retain)
                  0000af60    00000094     rti.obj (.text:retain)
                  0000aff4    00000094     rtsv7R4_T_be_v3D16_eabi.lib : auto_init.obj (.text)
                  0000b088    0000006c     sys_main.obj (.text)
                  0000b0f4    00000068     F021_API_CortexR4_BE.lib : Read.Common.obj (.text:_Fapi_enterMarginMode)
                  0000b15c    00000060     rtsv7R4_T_be_v3D16_eabi.lib : copy_decompress_rle.obj (.text)
                  0000b1bc    00000054                                 : u_div32.obj (.text)
                  0000b210    0000004c     F021_API_CortexR4_BE.lib : FlashStateMachine.EnableMainSectors.obj (.text:Fapi_enableMainBankSectors)
                  0000b25c    00000048     rtsv7R4_T_be_v3D16_eabi.lib : cpy_tbl.obj (.text)
                  0000b2a4    00000044                                 : exit.obj (.text)
                  0000b2e8    00000040     F021_API_CortexR4_BE.lib : Read.MarginByByte.obj (.text:Fapi_doMarginReadByByte)
                  0000b328    0000003c                              : FlashStateMachine.IssueFsmCommand.obj (.text:_Fapi_issueFsmCommand)
                  0000b364    00000036                              : Utilities.CalculateFletcher.obj (.text:Fapi_calculateFletcherChecksum)
                  0000b39a    00000002     --HOLE-- [fill = 0]
                  0000b39c    00000030                              : Async.WithAddress.obj (.text:Fapi_issueAsyncCommandWithAddress)
                  0000b3cc    00000030                              : Utilities.WaitDelay.obj (.text:Fapi_waitDelay)
                  0000b3fc    0000002c                              : Read.Common.obj (.text:_Fapi_exitMarginMode)
                  0000b428    00000022                              : Read.FlushPipeline.obj (.text:Fapi_flushPipeline)
                  0000b44a    0000001c                              : FlashStateMachine.InitializeFlashBanks.obj (.text:_Fapi_divideUnsignedLong)
                  0000b466    00000002     --HOLE-- [fill = 0]
                  0000b468    00000014                              : Utilities.CalculateEcc.obj (.text:Fapi_calculateEcc)
                  0000b47c    00000014     rtsv7R4_T_be_v3D16_eabi.lib : _lock.obj (.text)
                  0000b490    00000012                                 : copy_zero_init.obj (.text:decompress:ZI)
                  0000b4a2    00000002     --HOLE-- [fill = 0]
                  0000b4a4    00000010     F021_API_CortexR4_BE.lib : FlashStateMachine.ScaleFclk.obj (.text:_scaleEEFclk)
                  0000b4b4    00000010                              : FlashStateMachine.ScaleFclk.obj (.text:_scaleMainFclk)
                  0000b4c4    0000000e     rtsv7R4_T_be_v3D16_eabi.lib : copy_decompress_none.obj (.text:decompress:none)
                  0000b4d2    0000000c     F021_API_CortexR4_BE.lib : Read.WdService.obj (.text:_Fapi_checkWdService)
                  0000b4de    00000006     rtsv7R4_T_be_v3D16_eabi.lib : copy_decompress_rle.obj (.text:decompress:rle24)
                  0000b4e4    00000004     sys_phantom.obj (.text:retain)
                  0000b4e8    0000000a     Fapi_UserDefinedFunctions.obj (.tramp.Fapi_serviceWatchdogTimer.1)
                  0000b4f2    00000002     --HOLE-- [fill = 0]
                  0000b4f4    0000000c     bl_flash.obj (.tramp.Fapi_BlockProgram.1)
                  0000b500    0000000c     bl_flash.obj (.tramp.Fapi_BlockErase.1)
                  0000b50c    0000000c     bl_flash.obj (.tramp.BLInternalFlashStartAddrCheck.1)

.const     0    0000b518    0000035e     
                  0000b518    00000200     sys_vim.obj (.const:s_vim_init)
                  0000b718    00000140     bl_flash.obj (.const:flash_sector)
                  0000b858    00000014     bl_flash.obj (.const)
                  0000b86c    0000000a     bl_uart.obj (.const:.string)

.cinit     0    0000b878    00000050     
                  0000b878    0000002a     (.cinit..data.load) [load image, compression = rle]
                  0000b8a2    00000002     --HOLE-- [fill = 0]
                  0000b8a4    0000000c     (__TI_handler_table)
                  0000b8b0    00000008     (.cinit..bss.load) [load image, compression = zero_init]
                  0000b8b8    00000010     (__TI_cinit_table)

.data      0    080029e4    0000044c     UNINITIALIZED
                  080029e4    00000400     bl_uart.obj (.data:tab_1024)
                  08002de4    0000002e     sys_main.obj (.data)
                  08002e12    00000001     F021_API_CortexR4_BE.lib : FlashStateMachine.SetActiveBank.obj (.data)
                  08002e13    00000001     --HOLE--
                  08002e14    00000008                              : FlashStateMachine.ScaleFclk.obj (.data)
                  08002e1c    00000008     rtsv7R4_T_be_v3D16_eabi.lib : _lock.obj (.data)
                  08002e24    00000008                                 : exit.obj (.data)
                  08002e2c    00000004     bl_ymodem.obj (.data)

.bss       0    08002e30    000000f4     UNINITIALIZED
                  08002e30    00000078     spi.obj (.bss:g_spiPacket_t)
                  08002ea8    00000040     bl_ymodem.obj (.bss:file_name)
                  08002ee8    00000028     sci.obj (.bss:g_sciTransfer_t)
                  08002f10    0000000c     (.common:num_str$1)
                  08002f1c    00000004     (.common:JumpAddress)
                  08002f20    00000004     (.common:g_ulTransferAddress)


LINKER GENERATED COPY TABLES

__TI_cinit_table @ 0000b8b8 records: 2, size/record: 8, table size: 16
	.data: load addr=0000b878, load size=0000002a bytes, run addr=080029e4, run size=0000044c bytes, compression=rle
	.bss: load addr=0000b8b0, load size=00000008 bytes, run addr=08002e30, run size=000000f4 bytes, compression=zero_init


LINKER GENERATED HANDLER TABLE

__TI_handler_table @ 0000b8a4 records: 3, size/record: 4, table size: 12
	index: 0, handler: __TI_decompress_rle24
	index: 1, handler: __TI_decompress_none
	index: 2, handler: __TI_zero_init

VENEERS

callee name               veneer name
   callee addr  veneer addr  call addr  call info
--------------  -----------  ---------  ----------------
Fapi_doMarginReadByByte   $Ven$AT$L$PI$$Fapi_doMarginReadByByte
   0000b2e9     080029a8     080027cc   bl_flash.obj (.text)
Fapi_issueAsyncCommandWithAddress  $Ven$AT$L$PI$$Fapi_issueAsyncCommandWithAddress
   0000b39d     080029b4     0800233c   bl_flash.obj (.text)
Fapi_enableMainBankSectors  $Ven$AT$L$PI$$Fapi_enableMainBankSectors
   0000b211     080029c0     08002308   bl_flash.obj (.text)
                             08002504   bl_flash.obj (.text)
Fapi_setActiveFlashBank   $Ven$AT$L$PI$$Fapi_setActiveFlashBank
   0000a769     080029cc     080022d8   bl_flash.obj (.text)
                             080024fc   bl_flash.obj (.text)
                             08002644   bl_flash.obj (.text)
Fapi_initializeFlashBanks  $Ven$AT$L$PI$$Fapi_initializeFlashBanks
   0000a1cd     080029d8     080022c4   bl_flash.obj (.text)
                             080024f4   bl_flash.obj (.text)
                             0800263c   bl_flash.obj (.text)
                             080027b0   bl_flash.obj (.text)
Fapi_serviceWatchdogTimer  $Ven$TA$L$PI$$Fapi_serviceWatchdogTimer
   08002000     0000b4e8     0000b4d8   F021_API_CortexR4_BE.lib : Read.WdService.obj (.text:_Fapi_checkWdService)

[6 trampolines]
[12 trampoline calls]


FAR CALL TRAMPOLINES

callee name               trampoline name
   callee addr  tramp addr   call addr  call info
--------------  -----------  ---------  ----------------
Fapi_calculateEcc         $Tramp$TT$L$PI$$Fapi_calculateEcc
   0000b469     08002990     08002964   F021_API_CortexR4_BE.lib : Program.obj (.text:Fapi_issueProgrammingCommand)
_Fapi_issueFsmCommand     $Tramp$TT$L$PI$$_Fapi_issueFsmCommand
   0000b329     0800299c     080028cc   F021_API_CortexR4_BE.lib : Program.obj (.text:Fapi_issueProgrammingCommand)
                             0800297a                            : Program.obj (.text:Fapi_issueProgrammingCommand)
Fapi_BlockProgram         $Tramp$AA$L$PI$$Fapi_BlockProgram
   08002420     0000b4f4     00005f38   bl_ymodem.obj (.text)
                             0000607c   bl_ymodem.obj (.text)
Fapi_BlockErase           $Tramp$AA$L$PI$$Fapi_BlockErase
   08002134     0000b500     00005ea4   bl_ymodem.obj (.text)
BLInternalFlashStartAddrCheck  $Tramp$AA$L$PI$$BLInternalFlashStartAddrCheck
   08002058     0000b50c     00005e60   bl_ymodem.obj (.text)

[5 trampolines]
[7 trampoline calls]


GLOBAL SYMBOLS: SORTED ALPHABETICALLY BY Name 

address    name
--------   ----
08002008   BLInternalFlashFirstSectorSizeGet
08002030   BLInternalFlashSizeGet
08002058   BLInternalFlashStartAddrCheck
0000b2a5   C$$EXIT
08002134   Fapi_BlockErase
08002420   Fapi_BlockProgram
08002758   Fapi_BlockRead
080025f0   Fapi_UpdateStatusProgram
0000b469   Fapi_calculateEcc
0000b365   Fapi_calculateFletcherChecksum
0000b2e9   Fapi_doMarginReadByByte
0000b211   Fapi_enableMainBankSectors
0000b429   Fapi_flushPipeline
0000a1cd   Fapi_initializeFlashBanks
0000b39d   Fapi_issueAsyncCommandWithAddress
08002819   Fapi_issueProgrammingCommand
08002000   Fapi_serviceWatchdogTimer
0000a769   Fapi_setActiveFlashBank
0000b3cd   Fapi_waitDelay
08002e2c   FlashDestination
0800270c   Flash_Erase_Check
080026b4   Flash_Program_Check
00008040   Int2Str
08002f1c   JumpAddress
UNDEFED    SHT$$INIT_ARRAY$$Base
UNDEFED    SHT$$INIT_ARRAY$$Limit
00008134   Str2Int
000085fc   U32toStr
00008ef4   UART_Download
00009008   UART_Upload
000084ec   UART_getChar
000084b0   UART_getKey
00008768   UART_putChar
00008728   UART_putString
00008550   UART_rxByte
00008688   UART_send32BitData
000085c8   UART_txByte
000090f0   UpdaterUART
00005c4c   Ymodem_Receive
000063fc   Ymodem_Transmit
0000b4d3   _Fapi_checkWdService
0000b0f5   _Fapi_enterMarginMode
0000b3fd   _Fapi_exitMarginMode
0000b329   _Fapi_issueFsmCommand
0000b8b8   __TI_CINIT_Base
0000b8c8   __TI_CINIT_Limit
0000b8a4   __TI_Handler_Table_Base
0000b8b0   __TI_Handler_Table_Limit
000005bc   __TI_PINIT_Base
000005c0   __TI_PINIT_Limit
0000aff5   __TI_auto_init
08002e24   __TI_cleanup_ptr
0000b4c5   __TI_decompress_none
0000b4df   __TI_decompress_rle24
08002e28   __TI_dtors_ptr
00000000   __TI_static_base__
0000b491   __TI_zero_init
0000ae2d   __aeabi_memcpy
0000ae2d   __aeabi_memcpy4
0000ae2d   __aeabi_memcpy8
0000b1bc   __aeabi_uidivmod
ffffffff   __binit__
ffffffff   __c_args__
000005c4   _c_int00
000004b4   _coreClearAuxiliaryDataFault_
000004d0   _coreClearAuxiliaryInstructionFault_
0000047c   _coreClearDataFaultAddress_
00000444   _coreClearDataFault_
00000498   _coreClearInstructionFaultAddress_
00000460   _coreClearInstructionFault_
000003a8   _coreDisableEventBusExport_
0000040c   _coreDisableFlashEcc_
000003d8   _coreDisableRamEcc_
00000390   _coreEnableEventBusExport_
000003f0   _coreEnableFlashEcc_
00000424   _coreEnableIrqVicOffset_
000003c0   _coreEnableRamEcc_
00000378   _coreEnableVfp_
000004ac   _coreGetAuxiliaryDataFault_
000004c8   _coreGetAuxiliaryInstructionFault_
00000474   _coreGetDataFaultAddress_
0000043c   _coreGetDataFault_
00000490   _coreGetInstructionFaultAddress_
00000458   _coreGetInstructionFault_
00000200   _coreInitRegisters_
0000030c   _coreInitStackPointer_
0000aca0   _dabort
000004ec   _disable_FIQ_interrupt_
000004f4   _disable_IRQ_interrupt_
000004e4   _disable_interrupt_
000004fc   _enable_interrupt_
0000058c   _errata_CORTEXR4_57_
000005a4   _errata_CORTEXR4_66_
00000504   _esmCcmErrorsClear_
00000358   _getCPSRValue_
00000360   _gotoCPUIdle_
08002e1c   _lock
00009e98   _mpuAreRegionsSeparate_
00009e74   _mpuDisableBackgroundRegion_
00009e3c   _mpuDisable_
00009e5c   _mpuEnableBackgroundRegion_
00009e1c   _mpuEnable_
00009e8c   _mpuGetNumberOfRegions_
00009ebc   _mpuGetRegionBaseAddress_
00009edc   _mpuGetRegionPermission_
00009ed0   _mpuGetRegionType_
00009eac   _mpuGetRegion_
00009bf0   _mpuInit_
00009eb4   _mpuSetRegionBaseAddress_
00009ee8   _mpuSetRegionSizeRegister_
00009ec4   _mpuSetRegionTypeAndPermission_
00009ea4   _mpuSetRegion_
0000b48b   _nop
0000abf4   _pmuDisableCountersGlobal_
0000abdc   _pmuEnableCountersGlobal_
0000ac74   _pmuGetCycleCount_
0000ac7c   _pmuGetEventCount_
0000ac8c   _pmuGetOverflow_
0000ab8c   _pmuInit_
0000ac3c   _pmuResetCounters_
0000ac0c   _pmuResetCycleCounter_
0000ac24   _pmuResetEventCounters_
0000ac64   _pmuSetCountEvent_
0000ac54   _pmuStartCounters_
0000ac5c   _pmuStopCounters_
0000b483   _register_lock
0000b47d   _register_unlock
0000b4a5   _scaleEEFclk
0000b4b5   _scaleMainFclk
08002e20   _unlock
0000b2a9   abort
0000ad88   adc1Group1Interrupt
0000add4   adc1Group2Interrupt
0000342c   adc1ParityCheck
000034f4   adc2ParityCheck
0000a494   adcNotification
00001200   api_load
08002000   api_run
000009e4   api_size
ffffffff   binit
000035d0   can1ParityCheck
000036a8   can2ParityCheck
00003770   can3ParityCheck
0000a4a8   canErrorNotification
0000a4d0   canMessageNotification
0000a4bc   canStatusChangeNotification
00002210   ccmSelfCheck
000048cc   ccmr4GetConfigValue
00002af8   checkB0RAMECC
00002ce8   checkB1RAMECC
00003dd8   checkClockMonitor
00002ed8   checkFlashECC
00003eb4   checkFlashEEPROMECC
0000404c   checkPLL1Slip
0000414c   checkPLL2Slip
00004210   checkRAMAddrParity
00003b90   checkRAMECC
00004330   checkRAMUERRTest
0000297c   checkefcSelfTest
0000b25d   copy_in
00002414   cpuSelfTest
00002fbc   cpuSelfTestFail
00002fb4   custom_dabort
00004d28   disableParity
0000a5bc   dmaGroupANotification
0000306c   dmaParityCheck
0000a5d0   ecap1Interrupt
0000a648   ecap2Interrupt
0000a6c0   ecap3nterrupt
0000a5a8   ecapNotification
0000a55c   edgeNotification
00002820   efcCheck
00004834   efcGetConfigValue
00002954   efcSelfTest
000028a8   efcStuckZeroTest
00004ca0   enableParity
0000493c   errata_PBIST_4
0000976c   esmActivateNormalOperation
00009858   esmClearStatus
00009898   esmClearStatusBuffer
00009730   esmDisableError
000097a8   esmDisableInterrupt
00009704   esmEnableError
0000977c   esmEnableInterrupt
000099b8   esmEnterSelfTest
000096e8   esmError
00009a90   esmGetConfigValue
000098e4   esmGetStatus
00009958   esmGetStatusBuffer
0000a42c   esmGroup1Notification
0000a43c   esmGroup2Notification
0000a8e4   esmHighInterrupt
000095bc   esmInit
00009a40   esmSelfTestStatus
000098c4   esmSetCounterPreloadValue
000097d4   esmSetInterruptLevel
0000975c   esmTriggerErrorPinReset
0000a584   etpwmNotification
0000a594   etpwmTripNotification
0000b2b1   exit
08002ea8   file_name
0000b858   flash_bank
0000b718   flash_sector
00004494   fmcBus1ParityCheck
00002a1c   fmcBus2Check
00002a58   fmcECCcheck
08002de4   g_pulUpdateSuccess
08002f20   g_ulTransferAddress
08002e0c   g_ulUpdateBufferSize
08002e04   g_ulUpdateStatusAddr
08002e08   g_ulVectorTable
0000aa50   get_hardware_Info
0000aa3c   get_software_Version
0000aec8   gioHighLevelInterrupt
0000a4e4   gioNotification
00003118   het1ParityCheck
00003280   het2ParityCheck
0000a570   hetNotification
000031c4   htu1ParityCheck
0000337c   htu2ParityCheck
0000a4f8   i2cNotification
08002e10   iTimerForEEPROM
0000b088   main
00005008   mapClocks
0000ae2d   memcpy
00002354   memoryInit
0000a44c   memoryPort0TestFailNotification
0000a468   memoryPort1TestFailNotification
0000787c   mibspi1HighLevelInterrupt
00003844   mibspi1ParityCheck
0000394c   mibspi3ParityCheck
00007d4c   mibspi5HighLevelInterrupt
00007ae4   mibspi5LowLevelInterrupt
00003a70   mibspi5ParityCheck
00006f4c   muxInit
000045c0   pbistFail
00004640   pbistGetConfigValue
00002788   pbistIsTestCompleted
000027a4   pbistIsTestPassed
000027d8   pbistPortTestStatus
0000268c   pbistRun
000024ac   pbistSelfCheck
00002758   pbistStop
00004fb4   periphInit
0000b4e4   phantomInterrupt
00007448   pinmuxGetConfigValue
0000a544   pwmNotification
00000000   resetEntry
0000af60   rtiCompare2Interrupt
0000afa8   rtiCompare3Interrupt
0000a484   rtiNotification
00008c54   sciDisableLoopback
00008ce0   sciDisableNotification
00008c20   sciEnableLoopback
00008c78   sciEnableNotification
00008d48   sciGetConfigValue
000087a8   sciInit
00008ad0   sciIsIdleDetected
00008ab4   sciIsRxReady
00008934   sciIsTxReady
0000a50c   sciNotification
00008b48   sciReceive
00008b1c   sciReceiveByte
00008aec   sciRxError
00008980   sciSend
00008950   sciSendByte
000088b4   sciSetBaudrate
00008894   sciSetFunctional
00002200   selftestFailNotification
00006294   send_dataPacket
00004f74   setupFlash
00004ecc   setupPLL
0000a534   spiEndNotification
0000a520   spiNotification
000057ec   sramGetConfigValue
0000478c   stcGetConfigValue
00002398   stcSelfCheck
00002fb8   stcSelfCheckFail
0000522c   systemGetConfigValue
00005130   systemInit
000051fc   systemPowerDown
080029e4   tab_1024
00005640   tcmflashGetConfigValue
00004f2c   trimLPO
000065d0   vimChannelMap
00006834   vimDisableInterrupt
0000666c   vimEnableInterrupt
000068e0   vimGetConfigValue
000064fc   vimInit
00002fc0   vimParityCheck
00009ef0   vimParityErrorHandler


GLOBAL SYMBOLS: SORTED BY Symbol Address 

address    name
--------   ----
00000000   __TI_static_base__
00000000   resetEntry
00000200   _coreInitRegisters_
0000030c   _coreInitStackPointer_
00000358   _getCPSRValue_
00000360   _gotoCPUIdle_
00000378   _coreEnableVfp_
00000390   _coreEnableEventBusExport_
000003a8   _coreDisableEventBusExport_
000003c0   _coreEnableRamEcc_
000003d8   _coreDisableRamEcc_
000003f0   _coreEnableFlashEcc_
0000040c   _coreDisableFlashEcc_
00000424   _coreEnableIrqVicOffset_
0000043c   _coreGetDataFault_
00000444   _coreClearDataFault_
00000458   _coreGetInstructionFault_
00000460   _coreClearInstructionFault_
00000474   _coreGetDataFaultAddress_
0000047c   _coreClearDataFaultAddress_
00000490   _coreGetInstructionFaultAddress_
00000498   _coreClearInstructionFaultAddress_
000004ac   _coreGetAuxiliaryDataFault_
000004b4   _coreClearAuxiliaryDataFault_
000004c8   _coreGetAuxiliaryInstructionFault_
000004d0   _coreClearAuxiliaryInstructionFault_
000004e4   _disable_interrupt_
000004ec   _disable_FIQ_interrupt_
000004f4   _disable_IRQ_interrupt_
000004fc   _enable_interrupt_
00000504   _esmCcmErrorsClear_
0000058c   _errata_CORTEXR4_57_
000005a4   _errata_CORTEXR4_66_
000005bc   __TI_PINIT_Base
000005c0   __TI_PINIT_Limit
000005c4   _c_int00
000009e4   api_size
00001200   api_load
00002200   selftestFailNotification
00002210   ccmSelfCheck
00002354   memoryInit
00002398   stcSelfCheck
00002414   cpuSelfTest
000024ac   pbistSelfCheck
0000268c   pbistRun
00002758   pbistStop
00002788   pbistIsTestCompleted
000027a4   pbistIsTestPassed
000027d8   pbistPortTestStatus
00002820   efcCheck
000028a8   efcStuckZeroTest
00002954   efcSelfTest
0000297c   checkefcSelfTest
00002a1c   fmcBus2Check
00002a58   fmcECCcheck
00002af8   checkB0RAMECC
00002ce8   checkB1RAMECC
00002ed8   checkFlashECC
00002fb4   custom_dabort
00002fb8   stcSelfCheckFail
00002fbc   cpuSelfTestFail
00002fc0   vimParityCheck
0000306c   dmaParityCheck
00003118   het1ParityCheck
000031c4   htu1ParityCheck
00003280   het2ParityCheck
0000337c   htu2ParityCheck
0000342c   adc1ParityCheck
000034f4   adc2ParityCheck
000035d0   can1ParityCheck
000036a8   can2ParityCheck
00003770   can3ParityCheck
00003844   mibspi1ParityCheck
0000394c   mibspi3ParityCheck
00003a70   mibspi5ParityCheck
00003b90   checkRAMECC
00003dd8   checkClockMonitor
00003eb4   checkFlashEEPROMECC
0000404c   checkPLL1Slip
0000414c   checkPLL2Slip
00004210   checkRAMAddrParity
00004330   checkRAMUERRTest
00004494   fmcBus1ParityCheck
000045c0   pbistFail
00004640   pbistGetConfigValue
0000478c   stcGetConfigValue
00004834   efcGetConfigValue
000048cc   ccmr4GetConfigValue
0000493c   errata_PBIST_4
00004ca0   enableParity
00004d28   disableParity
00004ecc   setupPLL
00004f2c   trimLPO
00004f74   setupFlash
00004fb4   periphInit
00005008   mapClocks
00005130   systemInit
000051fc   systemPowerDown
0000522c   systemGetConfigValue
00005640   tcmflashGetConfigValue
000057ec   sramGetConfigValue
00005c4c   Ymodem_Receive
00006294   send_dataPacket
000063fc   Ymodem_Transmit
000064fc   vimInit
000065d0   vimChannelMap
0000666c   vimEnableInterrupt
00006834   vimDisableInterrupt
000068e0   vimGetConfigValue
00006f4c   muxInit
00007448   pinmuxGetConfigValue
0000787c   mibspi1HighLevelInterrupt
00007ae4   mibspi5LowLevelInterrupt
00007d4c   mibspi5HighLevelInterrupt
00008040   Int2Str
00008134   Str2Int
000084b0   UART_getKey
000084ec   UART_getChar
00008550   UART_rxByte
000085c8   UART_txByte
000085fc   U32toStr
00008688   UART_send32BitData
00008728   UART_putString
00008768   UART_putChar
000087a8   sciInit
00008894   sciSetFunctional
000088b4   sciSetBaudrate
00008934   sciIsTxReady
00008950   sciSendByte
00008980   sciSend
00008ab4   sciIsRxReady
00008ad0   sciIsIdleDetected
00008aec   sciRxError
00008b1c   sciReceiveByte
00008b48   sciReceive
00008c20   sciEnableLoopback
00008c54   sciDisableLoopback
00008c78   sciEnableNotification
00008ce0   sciDisableNotification
00008d48   sciGetConfigValue
00008ef4   UART_Download
00009008   UART_Upload
000090f0   UpdaterUART
000095bc   esmInit
000096e8   esmError
00009704   esmEnableError
00009730   esmDisableError
0000975c   esmTriggerErrorPinReset
0000976c   esmActivateNormalOperation
0000977c   esmEnableInterrupt
000097a8   esmDisableInterrupt
000097d4   esmSetInterruptLevel
00009858   esmClearStatus
00009898   esmClearStatusBuffer
000098c4   esmSetCounterPreloadValue
000098e4   esmGetStatus
00009958   esmGetStatusBuffer
000099b8   esmEnterSelfTest
00009a40   esmSelfTestStatus
00009a90   esmGetConfigValue
00009bf0   _mpuInit_
00009e1c   _mpuEnable_
00009e3c   _mpuDisable_
00009e5c   _mpuEnableBackgroundRegion_
00009e74   _mpuDisableBackgroundRegion_
00009e8c   _mpuGetNumberOfRegions_
00009e98   _mpuAreRegionsSeparate_
00009ea4   _mpuSetRegion_
00009eac   _mpuGetRegion_
00009eb4   _mpuSetRegionBaseAddress_
00009ebc   _mpuGetRegionBaseAddress_
00009ec4   _mpuSetRegionTypeAndPermission_
00009ed0   _mpuGetRegionType_
00009edc   _mpuGetRegionPermission_
00009ee8   _mpuSetRegionSizeRegister_
00009ef0   vimParityErrorHandler
0000a1cd   Fapi_initializeFlashBanks
0000a42c   esmGroup1Notification
0000a43c   esmGroup2Notification
0000a44c   memoryPort0TestFailNotification
0000a468   memoryPort1TestFailNotification
0000a484   rtiNotification
0000a494   adcNotification
0000a4a8   canErrorNotification
0000a4bc   canStatusChangeNotification
0000a4d0   canMessageNotification
0000a4e4   gioNotification
0000a4f8   i2cNotification
0000a50c   sciNotification
0000a520   spiNotification
0000a534   spiEndNotification
0000a544   pwmNotification
0000a55c   edgeNotification
0000a570   hetNotification
0000a584   etpwmNotification
0000a594   etpwmTripNotification
0000a5a8   ecapNotification
0000a5bc   dmaGroupANotification
0000a5d0   ecap1Interrupt
0000a648   ecap2Interrupt
0000a6c0   ecap3nterrupt
0000a769   Fapi_setActiveFlashBank
0000a8e4   esmHighInterrupt
0000aa3c   get_software_Version
0000aa50   get_hardware_Info
0000ab8c   _pmuInit_
0000abdc   _pmuEnableCountersGlobal_
0000abf4   _pmuDisableCountersGlobal_
0000ac0c   _pmuResetCycleCounter_
0000ac24   _pmuResetEventCounters_
0000ac3c   _pmuResetCounters_
0000ac54   _pmuStartCounters_
0000ac5c   _pmuStopCounters_
0000ac64   _pmuSetCountEvent_
0000ac74   _pmuGetCycleCount_
0000ac7c   _pmuGetEventCount_
0000ac8c   _pmuGetOverflow_
0000aca0   _dabort
0000ad88   adc1Group1Interrupt
0000add4   adc1Group2Interrupt
0000ae2d   __aeabi_memcpy
0000ae2d   __aeabi_memcpy4
0000ae2d   __aeabi_memcpy8
0000ae2d   memcpy
0000aec8   gioHighLevelInterrupt
0000af60   rtiCompare2Interrupt
0000afa8   rtiCompare3Interrupt
0000aff5   __TI_auto_init
0000b088   main
0000b0f5   _Fapi_enterMarginMode
0000b1bc   __aeabi_uidivmod
0000b211   Fapi_enableMainBankSectors
0000b25d   copy_in
0000b2a5   C$$EXIT
0000b2a9   abort
0000b2b1   exit
0000b2e9   Fapi_doMarginReadByByte
0000b329   _Fapi_issueFsmCommand
0000b365   Fapi_calculateFletcherChecksum
0000b39d   Fapi_issueAsyncCommandWithAddress
0000b3cd   Fapi_waitDelay
0000b3fd   _Fapi_exitMarginMode
0000b429   Fapi_flushPipeline
0000b469   Fapi_calculateEcc
0000b47d   _register_unlock
0000b483   _register_lock
0000b48b   _nop
0000b491   __TI_zero_init
0000b4a5   _scaleEEFclk
0000b4b5   _scaleMainFclk
0000b4c5   __TI_decompress_none
0000b4d3   _Fapi_checkWdService
0000b4df   __TI_decompress_rle24
0000b4e4   phantomInterrupt
0000b718   flash_sector
0000b858   flash_bank
0000b8a4   __TI_Handler_Table_Base
0000b8b0   __TI_Handler_Table_Limit
0000b8b8   __TI_CINIT_Base
0000b8c8   __TI_CINIT_Limit
08002000   Fapi_serviceWatchdogTimer
08002000   api_run
08002008   BLInternalFlashFirstSectorSizeGet
08002030   BLInternalFlashSizeGet
08002058   BLInternalFlashStartAddrCheck
08002134   Fapi_BlockErase
08002420   Fapi_BlockProgram
080025f0   Fapi_UpdateStatusProgram
080026b4   Flash_Program_Check
0800270c   Flash_Erase_Check
08002758   Fapi_BlockRead
08002819   Fapi_issueProgrammingCommand
080029e4   tab_1024
08002de4   g_pulUpdateSuccess
08002e04   g_ulUpdateStatusAddr
08002e08   g_ulVectorTable
08002e0c   g_ulUpdateBufferSize
08002e10   iTimerForEEPROM
08002e1c   _lock
08002e20   _unlock
08002e24   __TI_cleanup_ptr
08002e28   __TI_dtors_ptr
08002e2c   FlashDestination
08002ea8   file_name
08002f1c   JumpAddress
08002f20   g_ulTransferAddress
ffffffff   __binit__
ffffffff   __c_args__
ffffffff   binit
UNDEFED    SHT$$INIT_ARRAY$$Base
UNDEFED    SHT$$INIT_ARRAY$$Limit

[291 symbols]
